:0300000002349F28
:0C349F0078FFE4F6D8FD7581540234E695
:10137A0020000A3C2E2E2E3E004950436F6E6E65A9
:10138A0063745245510A004950436F6E6E65637427
:10139A00000A49504E6F41434B210A003E432C56E6
:1013AA002C52432CC0E4E0EFF2E5F020D1E8EDEA5C
:1013BA00EEEC49500A003E432C4D41432C25303275
:1013CA0062583A25303262583A25303262583A2504
:1013DA00303262583A25303262583A2530326258F1
:1013EA002C4D414320E0E4F0E5F10A003E432C563F
:1013FA0045522C20332E3220EEF2202573202573FD
:10140A002CC2E5F0F1E8FF20495020ECEEE4F3EBC2
:10141A00FF0A004A756C20313120323030380031F1
:10142A00363A35313A3130003E432C4C442C505236
:10143A004F473A2020202020202020202020202032
:10144A002020202020202020202020202020202092
:10145A002020202020202020202020202020202082
:10146A002020202020202020202020202020202072
:10147A0020202020202020202CC4E0F2E020EFF0C1
:10148A00EEF8E8E2EAE828F4E0E9EB290A003E2A65
:10149A002C312CCEF1EDEEE2EDFBE520EFE0F0E0B1
:1014AA00ECE5F2F0FB20F1E5F2E5E2EEE3EE20E80E
:1014BA00EDF2E5F0F4E5E9F1E00A003E412C4130B5
:1014CA00312C2562752E2562752E2562752E2562B0
:1014DA00752C495020E0E4F0E5F120E0E4E0EFF279
:1014EA00E5F0E00A003E412C4130322C2562752E8F
:1014FA002562752E2562752E2562752C495020E0CD
:10150A00E4F0E5F120EEF1ED2E20F1E5F0E2E5F070
:10151A00E00A003E412C4130332C2562752E2562AB
:10152A00752E2562752E2562752C495020E0E4F04F
:10153A00E5F120F0E5E72E20F1E5F0E2E5F0E00A3A
:10154A00003E412C4130342C2562752E2562752EC1
:10155A002562752E2562752CCCE0F1EAE020F1E5D2
:10156A00F2E80A003E412C4130352C2562752E25C1
:10157A0062752E2562752E2562752CD8EBFEE70A58
:10158A00003E2A2C312CC4EEEF2E20EFE0F0E0ECE6
:10159A00E5F2F0FB20F1E5F2E5E2EEE3EE20E8ED1C
:1015AA00F2E5F0F4E5E9F1E00A003E422C5330316D
:1015BA002C2562752CC6E4E0F2FC20E7E0EFF0EEA1
:1015CA00F1E020F1EEE5E4E8EDE5EDE8FF20EEF2EA
:1015DA0020F1E5F0E2E5F0E00A003E422C53303219
:1015EA002C2562752CCEE1ECE5ED20F120F1E5F039
:1015FA00E2E5F0EEEC20E1E5E720EAE2E8F2E0EDF0
:10160A00F6E8E90A003E422C5330332C2562752C49
:10161A00CFE5F0E5E7E0EFF3F1EA20EFF0E820EFBD
:10162A00EEF2E5F0E520F1E2FFE7E820F120F1E54E
:10163A00F0E2E5F0EEEC0A003E454E440A000A44A8
:10164A00756D705820202020203030203031203015
:10165A0032203033203034203035203036203037B5
:10166A002030382030392030412030422030432089
:10167A0030442030452030460A000A3A003A200019
:10168A000A000A44756D7044202020202030302042
:10169A003031203032203033203034203035203081
:1016AA00362030372030382030392030412030423F
:1016BA0020304320304420304520304600457272A5
:1016CA00206B657900526420656570726F6D0A003F
:1016DA005264204D454D0A00526420436F64650AE6
:1016EA0000577269746520436F64650A0044656235
:1016FA0075674950204F4E0A004465627567495024
:10170A00204F46460A004465627567557365722024
:10171A004F6E0A00446562756755736572204F46BD
:10172A00460A0044656275674D7367204F6E0A006A
:10173A0044656275674D7367204F46460A00436FDA
:10174A006E666967206C6F636B210A0057722065A9
:10175A006570726F6D0A0020536176652065657049
:10176A00726F6D210A00457272204D414321004C6F
:10177A006F61643E3E002A003C4130313D003C41ED
:10178A0030323D003C4130333D003C4130343D0075
:10179A003C4130353D003C21003C5330313D003C5A
:1017AA005330323D003C5330333D003C5330353DDD
:0717BA00003C5330363D00F6
:063D2900015100014F00F2
:103D7300C28E438910E4F58B758DB8D2ABD28E22F7
:03001B0002340F9D
:10340F00C0E0C083C082C0D0C28E758B00758DB8EE
:10341F00201D0675A61E75A6E1054FD219E5516050
:10342F00020551E550D39401400215500554E5545F
:10343F00540F7048D225E554543F7012D21790663E
:10344F008BE0600A04F0E0D394B44002D21D906682
:10345F0086E0600204F0906104E0600214F0906670
:10346F008CE0D394014003E014F0301C020552E5C8
:10347F0053D394644004D21D80020553E54ED39478
:10348F00014002154ED28ED0D0D082D083D0E03200
:1008CC00C2AFC2227D027C007F07123D0C8F26E551
:1008DC0026646060097D017F60123CA4D222E4FD95
:1008EC00FC7F0B123D0C8F26E52630E6097D04E4D7
:1008FC00FF123CC8D2227D017C007F07123D0C8F79
:10090C0026E5267008FD7FFF123CA4D2223022037C
:10091C00126000C288C2A8C2AA75890012337390F3
:10092C0063497403F0A374CCF0E4906348F0122F85
:10093C00E612316CC21D1239D4D222C224C22390C9
:10094C0065767408F09062B47424F0E4A3F09063BC
:10095C003EE09062B6F090633FE09062B7F0906337
:10096C0040E09062B8F0906341E09062B9F090631F
:10097C0042E09062BAF0906343E09062BBF0755035
:10098C0001E4906577F0C21EC21FC220C221202252
:10099C0018AF26FE7D03122E2AE4FF1232207E139E
:1009AC007F7AE4FBFDFC12294A90668BE0600374AD
:1009BC0001F0E4906104F0F552906575F0F5531276
:1009CC003D7375A70775A61E75A6E1D2AFE4F55366
:1009DC00906104E07003123A8490668CE0B40111CB
:1009EC009080007410F0E490668CF0D222C223C286
:1009FC0024908008E0F52630E405D21E7410F0E552
:100A0C002630E508D2209080087420F0E52630E6E8
:100A1C0008D21F9080087440F0E552C3940340192B
:100A2C00908002E4F0908001F0908000F0E5529408
:100A3C00064006E4F5521239D49080A0E0700312FF
:100A4C0037C79080B8E070031238419080D0E070C6
:100A5C00031238BB908000E07013301E10122A5124
:100A6C00906331EFF0D39400400312002690800283
:100A7C00E07006908000E06005D21C0209D9C21C0F
:100A8C00E4F552906104E060030209D9202212902F
:100A9C006578E0600C7E137F7C122D42E4906578C3
:100AAC00F0302012122690906331EFF0D394004076
:100ABC0005E0FF123DEB201F03020C3D12250990AF
:100ACC006331EFF070030209D9906375E054BF24D1
:100ADC007F7003020BA6147003020B7E24026003CA
:100AEC00020BDF2022077E137F83122D4220260368
:100AFC00020C3D90634DE0FF7006906351E0606125
:100B0C00906682E0FEB50722A3E0FF90634EE0B54D
:100B1C000718906684E0FF90634FE0B5070C906671
:100B2C0085E0FF906350E06F6037906351E06E603A
:100B3C0003020C3D906683E0FF906352E06F60030C
:100B4C00020C3D906684E0FF906353E06F600302FB
:100B5C000C3D906685E0FF906354E06F6003020CDF
:100B6C003DC21A9065777401F012001E7550010297
:100B7C000C3D90668BE060037401F090667AE0FFA8
:100B8C00906377E06F6003020C3D90667AE004F0AE
:100B9C00E4F550906575F0020C3D301A03020C3DE3
:100BAC00906344E070030209D9906355740AF01203
:100BBC003DD2D21AE4F550906575F090668604F03B
:100BCC00E4906679F0A3F02022677E137F91122DBA
:100BDC0042805E90668BE060037401F0301A529094
:100BEC006375E020E74B906377E0FF906679E0FE59
:100BFC006F600D906681E07007EE146F7033801398
:100C0C00906679E004F0906331E0FFD394044003E4
:100C1C00123A2D9060007482F0A37401F090637707
:100C2C00E0906002F07E607F007D031235B2020915
:100C3C00D9201A03020D55E5507068122375EF6028
:100C4C00237E647F75906476E02404FD1235B290A7
:100C5C006681E07009906355E0F5500209D9E4F51E
:100C6C00500209D9906686E0D3943C403690668158
:100C7C00E0703090668604F01230B0E4906475F049
:100C8C00A37412F090667AE0906477F0A374FDF090
:100C9C0090610563A20190647963A2017F12122016
:100CAC00C3809E123D928F26E526B40115906000FC
:100CBC007483F0E4A3F07E607F007D021235B202F3
:100CCC0009D9E526D39401401C9060007483F0A3ED
:100CDC007401F0E52624FEA3F07E607F007D0312F4
:100CEC0035B20209D9E550640160030209D9906557
:100CFC0075E004F02022077E137F9B122D42906337
:100D0C0055E0C394C85004E02432F0906575E0C3FC
:100D1C009405400DC21AE4906577F012001E02098A
:100D2C00D97C667D82906349E0FAA3E0FB7F0212D6
:100D3C0037437E647F75906476E02404FD1235B2EF
:100D4C00906355E0F5500209D9E550640160030247
:100D5C0009D9906577E014604624FE604214700354
:100D6C00020E48240460030209D9E4F5522026132C
:100D7C009065777404F0906575E05401F07550013E
:100D8C000209D99080027410F0E4906577F09065B8
:100D9C007504F07550FA90668274FFF00209D990D0
:100DAC006682E07003020E329064757480F0906479
:100DBC00777401F0E4A3F0A304F0A37430F0A374EF
:100DCC007BF0E4F526747C2526F582E43464F58307
:100DDC00747DF0747D2526F582E43464F583E4F0AB
:100DEC00E5262407906476F07C667D82906349E06A
:100DFC00FAA3E0FB7F021237437E647F75E526245D
:100E0C0009FD1235B2906681E0601B123DD2D21AF8
:100E1C00E4F550906575F090668604F0E490667980
:100E2C00F0A3F00209D9302607E4906577F080062C
:100E3C009065777404F07550FA0209D990800274A9
:100E4C0010F0755005906575E06401FFF0906577C2
:100E5C007401F0EF7019906351E06013FCA3E0FD96
:100E6C00A3E0FEA3E0FF906682121C620209D990F7
:100E7C00634DE0FCA3E0FDA3E0FEA3E0FF906682DF
:090E8C00121C620209D980FE2249
:10002600906376E0B444047F0180027F009063759C
:10003600E0B447047E0180027E00EE5F604A906372
:100046003EE0906377F090633FE0906378F09063D2
:1000560040E0906379F0906341E090637AF09063BA
:1000660042E090637BF0906343E090637CF09063A2
:10007600767452F09062AE63A2019080A863A201EA
:100086007F061220C30208C2906331E0C394085071
:10009600030208CB90633EE0FF906377E06F600356
:1000A6000208CB90633FE0FF906378E06F60030245
:1000B60008CB906340E0FF906379E06F600302082D
:1000C600CB906341E0FF90637AE06F60030208CB58
:1000D600906342E0FF90637BE06F60030208CB9081
:1000E6006343E0FF90637CE06F60030208CB90639C
:1000F60076E0B444159062AEE0B4FF0E63A20190C0
:1001060080A863A2017F061220C390668BE060037D
:100116007401F090668C7464F09063767452F0907B
:100126006375E0646D60030202537BFF7A1379A660
:100136001218237BFF7A1379C090633EE0F52FA354
:10014600E0F530A3E0F531A3E0F532A3E0F533A303
:10015600E0F534121823752FFF75301475311D75AF
:1001660032FF7533147534297BFF7A1379F612182A
:10017600237BFF7A1479321218237BFF7A1479983D
:100186001218237BFF7A1479C5906344E0F52FA3F8
:10019600E0F530A3E0F531A3E0F5321218237BFF3A
:1001A6007A1479EF90634DE0F52FA3E0F530A3E0E4
:1001B600F531A3E0F5321218237BFF7A15791D90ED
:1001C6006351E0F52FA3E0F530A3E0F531A3E0F5A8
:1001D600321218237BFF7A15794B90633AE0F52F9C
:1001E600A3E0F530A3E0F531A3E0F5321218237B46
:1001F600FF7A15796E906336E0F52FA3E0F530A30C
:10020600E0F531A3E0F5321218237BFF7A15798BDE
:100216001218237BFF7A1579B4A226E433F52F1240
:1002260018237BFF7A1579E4906681E0F52F121882
:10023600237BFF7A16790F90668BE0F52F12182331
:100246001232D07BFF7A16794212182322906375F8
:10025600E0644C60030203127E167F48FBFDFC122D
:10026600294A90637DE0F527A3E0F528E4F52AE422
:10027600F529852882852783E0FF747F2529F58265
:10028600E43463F583EFF00529E529B410E4E527A6
:1002960090637FF0A3E528F07E167F847C637D7FE4
:1002A6007B0212294AE4F529852882852783E0FF07
:1002B600747F2529F582E43463F583EFF00528E59C
:1002C60028700205270529E529B410DC7E167F87EC
:1002D6007C637D7F7B1012294AE4F5298528828577
:1002E6002783E0FF747F2529F582E43463F583EFE5
:1002F600F00529E529B410E4052AE52AC39410502F
:10030600030202757E167F8A122D4222906375E0E3
:10031600646C60030203B3F52B7E167F8CFBFDFC39
:1003260012294AE4F52AE4F529A82BE6FF747F256D
:1003360029F582E43463F583EFF00529E529B41045
:10034600E8E490637FF0A3E52BF07E167F847C6360
:100356007D7F7B0212294AE4F529A82BE6FF747FEC
:100366002529F582E43463F583EFF0052B0529E5AD
:1003760029B410E67E167F877C637D7F7B10122969
:100386004AE4F529A82BE6FF747F2529F582E43493
:1003960063F583EFF00529E529B410E8052AE52A77
:1003A600C3940840817E167F8A122D42229063757F
:1003B600E0644B7061F52974672529F582E434639E
:1003C600F583E0603274672529F582E43463F583AA
:1003D600E0F4602374672529F582E43463F583E04D
:1003E600FF747D2529F582E43463F583E0B50710B3
:1003F6000529E529B408C09061047432F00208C2E8
:100406009063757421F03022030208C27E167FC7FE
:10041600122D420208C2906375E0B4521A202207D8
:100426007E167FCF122D429063757472F07E637FC5
:10043600757D0812352B22906375E064497045205E
:1004460022077E167FDA122D4290637DE0F527A300
:10045600E0F528E4F529852882852783E0FF747F67
:100466002529F582E43463F583EFF00528E5287045
:100476000205270529E529B480DC7E637F757D8A20
:1004860012352B22906375E0644370462022077E66
:10049600167FE2122D4290637DE0F527A3E0F52852
:1004A600E4F529852882852783E493FF747F25292F
:1004B600F582E43463F583EFF00528E5287002053C
:1004C600270529E529B480DB7E637F757D8A123591
:1004D6002B22906375E0645A70532022077E167FA4
:1004E600EB122D4290637DE0F527A3E0F5287C63AF
:1004F6007D7F7B80AF28AE27123BCAE4F52985288D
:1005060082852783E493FF747F2529F582E434638B
:10051600F583EFF00528E528700205270529E5296A
:10052600B480DB7E637F757D8A12352B22906375DE
:10053600E0644460030205C490637DE0FF64447098
:10054600030208C2EFB4310CC2227E167FF7122DC9
:10055600420208C290637DE0B4300CD2227E177F3F
:1005660003122D420208C290637DE0B4320CD223FE
:100576007E177F10122D420208C290637DE0B433CD
:100586000CC2237E177F1E122D420208C290637D85
:10059600E0B4340CD2247E177F2D122D420208C2FD
:1005A60090637DE0B4350CC2247E177F3A122D424B
:1005B6000208C290637DE0FF123DEA0208C2906124
:1005C60004E070132022077E177F48122D429063A5
:1005D600757421F00208C29061047432F09063755C
:1005E600E0FFB45104C2AF80FEEF6457704520228D
:1005F600077E177F56122D4290637EE0906331F09E
:10060600E4F529906331E0FFE529C39F4003020822
:10061600C2747F2529F582E43463F583E0FF906395
:100626007DE0252924ADF582E43461F583EFF005FC
:100636002980D0906375E0645360030206E62022A9
:10064600077E177F61122D4290633EE0FF9061B6F0
:10065600E06F703C90633FE0FF9061B7E06F7030F1
:10066600906340E0FF9061B8E0B50724906341E0F5
:10067600FF9061B9E0B50718906342E0FF9061BA58
:10068600E0B5070C906343E0FF9061BBE06F601636
:100696009063757421F03022030208C27E177F70C2
:1006A600122D420208C2E4F529E4F55374AD25295A
:1006B600F582E43461F583E0FDAF29123C2A052971
:1006C600E529C394FE40E2C2AFE4907FF0F0A3F0C8
:1006D600907FFD74AAF0A374FFF0A37455F080FE1A
:1006E600906375E0644F704C90637DE0F527A3E05E
:1006F600F528E5284527700A2022077E177F7912FC
:100706002D422022077E177F80122D42E4F52974A0
:100716007F2529F582E43463F583E08528828527E1
:1007260083F00528E528700205270529E529B48008
:10073600DE0208C2906375E0FFB4452190637DE058
:10074600FDA3E0907FF0CDF0A3EDF0C2AF907FFD6A
:1007560074AAF0A374FFF0A37455F080FEEF6465ED
:1007660060030208CB90637DE0FFA3E0907FF0CFAB
:10077600F0A3EFF0E4F527F528D3907FF1E0952874
:10078600907FF0E095274021E4F5532528FFE527E3
:100796003478FE7B80AD28AC27123BCA74802528AE
:1007A600F528E43527F52780D07E177F8212363963
:1007B600EF4E6020120003906344EFF012000390A6
:1007C6006345EFF0120003906346EFF012000390CA
:1007D6006347EFF07E177F88123639EF4E6020129E
:1007E600000390634DEFF012000390634EEFF0129A
:1007F600000390634FEFF0120003906350EFF07E1A
:10080600177F8E123639EF4E602012000390635127
:10081600EFF0120003906352EFF01200039063535F
:10082600EFF0120003906354EFF07E177F941236B8
:1008360039EF4E602012000390633AEFF012000386
:1008460090633BEFF012000390633CEFF01200035D
:1008560090633DEFF07E177F9A123639EF4E602097
:10086600120003906336EFF0120003906337EFF047
:10087600120003906338EFF0120003906339EFF033
:10088600E4F529E4F553E52904FF74362529F582B4
:10089600E43463F583E0FD123C2A0529E529C39477
:1008A6004340E0C2AFE4907FF0F0A3F0907FFD7488
:1008B600AAF0A374FFF0A37455F080FE7E637F75E3
:0608C6007D0812352B2213
:103B5C00AE07EEC39430400BEED394395005EE24EF
:103B6C00D0FF22EEC39461400BEED394665005EE69
:103B7C0024A9FF22EEC39441400BEED3944650058A
:083B8C00EE24C9FF22AF06225E
:103D45009062ADE004F070069062ACE004F0906221
:0A3D5500ACE0FEA3E0FF123B1A22CF
:10000300123D45123B5CEFC454F0FEC006123D4561
:08001300123B5CD0E02FFF223C
:10391E00E49069C2F0123D459069C3EFF0C3943054
:10392E004018E0FFD3943950119069C2E02405F598
:10393E0082E43461F583EFF080119069C2E02405D2
:10394E00F582E43461F583E4F0800C9069C2E00402
:10395E00F0E0D3940840BE75320075330075340024
:0D396E00E4F5357B017A6179051221D12243
:103639008E2C8F2D9062ACE4F0A374FFF0123D45FF
:10364900EF606EF4606B852D82852C83E493B5075A
:10365900EC752E01E52D252EF582E4352CF583E454
:103669009360259062ADE0252EFF9062ACE03400B6
:10367900FE123B1AE52D252EF582E4352CF583E45F
:1036890093B50704052E80CCE52D252EF582E4356A
:103699002CF583E49370A6E52E24FFFFE434FFFEA6
:1036A9009062ADE02FF09062ACE03EF07E007F01C9
:0536B90022E4FEFF22E7
:102FE6007E177FA0123639EF4E70037F01227E17BF
:102FF6007FA3123639EF4E600C123D45EF24D024E4
:10300600FF92268002D2267E177FA9123639EF4E0E
:10301600600C123D45EF24D0906681F08005E49067
:103026006681F07E177FAF123639EF4E600C123D87
:1030360045EF24D090668BF08005E490668BF07E99
:10304600177FB5123639EF4E600C123D45EF24D08E
:1030560024FF92188002C21890633E63A201906614
:103066007B63A2017F061220C330183B7E177FBB0D
:10307600123639EF4E603012000390667BEFF01285
:10308600000390667CEFF012000390667DEFF0126D
:10309600000390667EEFF012000390667FEFF01259
:0A30A6000003906680EFF07F002227
:103AD300906576E0C3947C503D906576E0FE04F0FB
:103AE30074B42EF582E43462F583EFF0BF0A2790B5
:103AF3006576E0FF04F074B42FF582E43462F58355
:103B0300E4F0906576E0FF1236BE9065767408F0B7
:073B13009062B5E004F0220E
:100E95005452414E5A0053545245414D00525453F9
:100EA5000044454C4159004D4F4445004C494D497E
:100EB500540053495A45004C454E47544800455641
:100EC500454E504152495459004F444450415249AE
:100ED5005459004B56545F494E004B56545F4F557D
:100EE5005400574149540053544F5000003E2A2C9A
:100EF500312CCFE0F0E0ECE5F2F0FB20E0F1E8ED9D
:100F0500F5F0EEEDEDEEE3EE20EFEEF0F2E02E2063
:100F1500D0E5E6E8EC20F0E0E1EEF2FB202D20EF55
:100F2500E0EAE5F2EDFBE90A003E4C2C4930312CB4
:100F3500256C752CD1EAEEF0EEF1F2FC20EEE1EC39
:100F4500E5EDE02C35302C3130302C3330302C367B
:100F550030302C313230302C323430302C34383083
:100F6500302C393630302C31393230302C3338345E
:100F750030302C35373630302C3131353230300A7F
:100F8500003E422C4930322C2562752CD3EFF0E01F
:100F9500E2EBE5EDE8E520EFEEF2EEEAEEEC20EF30
:100FA500F0E820EFE5F0E5E4E0F7E52028525453BA
:100FB5002D435453290A003E532C4930332C2562C6
:100FC500752CC7E0E4E5F0E6EAE020F1F2E0F0F2A6
:100FD500E020EFE5F0E5E4E0F7E8282A3130ECF130
:100FE500290A003E422C4930342C2562752CD0E567
:100FF500E6E8EC20EFE5F0E5E4E0F7E8203720E16E
:10100500E8F20A003E422C4930352C2562752CCF7A
:10101500E5F0E5E4E0F7E020F120EAEEEDF2F0EEB0
:10102500EBFCEDFBEC20E1E8F2EEEC0A003E422C95
:101035004930362C2562752CCAEEEDF2F0EEEBFC4C
:10104500EDFBE920E1E8F2202D20F7E5F2EDEEF1E8
:10105500F2FC0A003E422C415030372C2562752C9B
:10106500C6E4E0F2FC20EAE2E8F2E0EDF6E8FE2074
:10107500EEF220F3F1F2F0EEE9F1F2E2E00A003EE1
:10108500422C415030382C2562752CCAE2E8F2E832
:10109500F0EEE2E0F2FC20EFE0EAE5F2FB20EEF212
:1010A50020F3F1F2F0EEE9F1F2E2E00A003C210072
:1010B5003C4930313D003C4930323D003C493033FC
:1010C5003D003C4930343D003C4930353D003C490C
:1010D50030363D003C415030373D003C41503038C2
:1010E5003D000A53656E64205061636B65743A2058
:1010F500000A53656E64204B56543A20000AC1F32A
:10110500F4E5F020E7E0EDFFF221000A4352432029
:101115006572726F7221202020000ACEF2E2E5F797
:10112500E0FE20EDE020E7E0E3F0F3E7EAF321005D
:101135000A526563204B5654000A526563206F6B53
:101145002120202020202000FF0E95FF0E9BFF0E62
:10115500A2FF0EA6FF0EACFF0EB1FF0EB7FF0EBC31
:10116500FF0EC3FF0ECEFF0ED8FF0EDFFF0EE7FF0B
:101175000EECFF0EF100112332465765748C9DAFBE
:10118500BECADBE9F810013322564775649C8DBF52
:10119500AEDACBF9E82130021367764455ADBC8E43
:1011A5009FEBFAC8D93120120377665445BDAC9E32
:1011B5008FFBEAD8C94253617004152736CEDFED9F
:1011C500FC8899ABBA5243716014053726DECFFD12
:1011D500EC9889BBAA6372405125340617EFFECC03
:1011E500DDA9B88A9B7362504135241607FFEEDCF2
:1011F500CDB9A89A8B8495A7B6C2D3E1F008192B6F
:101205003A4E5F6D7C9485B7A6D2C3F1E018093BD1
:101215002A5E4F7D6CA5B48697E3F2C0D129380AC2
:101225001B6F7E4C5DB5A49687F3E2D0C139281AB1
:101235000B7F6E5C4DC6D7E5F48091A3B24A5B691E
:10124500780C1D2F3ED6C7F5E49081B3A25A4B7991
:10125500681C0D3F2EE7F6C4D5A1B082936B7A4882
:10126500592D3C0E1FF7E6D4C5B1A092837B6A5871
:10127500493D2C1E0F0089129B24AD36BF48C15A2B
:10128500D36CE57EF78108931AA52CB73EC940DBE0
:1012950052ED64FF76028B109926AF34BD4AC358D0
:1012A500D16EE77CF5830A9118A72EB53CCB42D9C0
:1012B50050EF66FD74048D169F20A932BB4CC55EA8
:1012C500D768E17AF3850C971EA128B33ACD44DFA0
:1012D50056E960FB72068F149D22AB30B94EC75C90
:1012E500D56AE378F1870E951CA32AB138CF46DD80
:1012F50054EB62F97008811A932CA53EB740C95288
:10130500DB64ED76FF89009B12AD24BF36C148D35F
:101315005AE56CF77E0A8318912EA73CB542CB504F
:10132500D966EF74FD8B029910AF26BD34C34AD13F
:1013350058E76EF57C0C851E9728A13AB344CD5627
:10134500DF60E972FB8D049F16A920BB32C54CD71F
:101355005EE168F37A0E871C952AA338B146CF540F
:10136500DD62EB70F98F069D14AB22B930C74ED5FF
:051375005CE36AF17861
:103D2F0052668D000000000000000000000000003F
:053D3F0000000000007F
:013DEA0022B6
:03002300022C515B
:102C5100C0E0C083C082C0D075D01830986775516C
:102C610001AF9920020CEF64027058750905D20278
:102C71008051300F14C20FAE0E050E74AE2EF582C8
:102C8100E43467F583EFF08037BF0904D20F803059
:102C9100BF0205530E808028BF03159067ACE50E77
:102CA100F0630E80530E80C202D2087509008010B5
:102CB100AE0E050E74AE2EF582E43467F583EFF0A7
:102CC100750905C29830996E300369301007309745
:102CD10004D200805F9066A1E0FFE510C39F400F22
:102CE100C203D213200B02D215C20BD2968045AF7C
:102CF10010051074AE2FF582E43468F583E0F51108
:102D010030091953117F30012820D0082004226393
:102D11001180801D30041A6311808015300112E585
:102D2100115211300406A2D0929B8005A2D0B39219
:102D31009B851199C299D2AFD0D0D082D083D0E0F7
:012D4100325F
:10397B008F2F9067ADE0FF04F074A22FF582E43433
:10398B0066F5837420F0E4FFEFC39D503BE52F7584
:10399B00F003A4244DF582E43411F583E493FB7416
:1039AB000193FA740293F98F82758300121B36FE12
:1039BB009067ADE024A2F582E43466F583EEF00F58
:0939CB009067ADE004F080C02219
:103C7D00742D2FF582E43461F583E0FE6420601627
:103C8D009067ADE0FD04F074A22DF582E43466F585
:073C9D0083EEF00F80DA2234
:101D8E00C209C204C201C212C210D20CE4F50AD2B8
:101D9E00139069AE74FFF0A374B8F0C20AC205C204
:101DAE0011E4F50DF50FF527E52775F003A4244D85
:101DBE00F582E43411F583E493FB740193FA740213
:101DCE0093F9121B1D7003021FE7E4F529F52AF59E
:101DDE0028742D2528F582E43461F583E0FF700325
:101DEE00021FE2E52775F003A4244DF582E43411B9
:101DFE00F583E493FB740193FA740293F9852982B7
:101E0E00758300121B36FEEFB50608752A010529EB
:101E1E00021FDDE52A7003021FDDEE6003021FD8EC
:101E2E00AD29AF2712397BE527B40E004003021F00
:101E3E00E2901E46F8282873021E70021EBC021E77
:101E4E00C1021EC6021EF8021F31021F31021F31CF
:101E5E00021F62021F68021F6C021F72021F7802AD
:101E6E001FA8AF28123C7D742D2528F9E43461FAA1
:101E7E007B01C0031B8B32753300753400E4F535DE
:101E8E00D0031221D18F2E8E2D8D2C8C2BAB2EAA02
:101E9E002DA92CA82B7F007E8C7D0A7C00121BB1F5
:101EAE00121C439069AEEEF0A3EFF0021FE2C20CDB
:101EBE00021FE2D210021FE2AF28123C7D742D25C4
:101ECE0028F9E43461FA7B01C0031B8B32753300B1
:101EDE00753400E4F535D0031221D18F2E8E2D8D61
:101EEE002C8C2BAF2E8F0A021FE2AF28123C7D7472
:101EFE002D2528F582E43461F583E0B43702D2094A
:101F0E00742E2528F582E43461F583E0FFB44E0487
:101F1E00C2018002D201EF64456003021FE2D204C7
:101F2E00021FE2AF28123C7D742D2528F9E434619E
:101F3E00FA7B01C0031B8B32753300753400E4F558
:101F4E0035D0031221D18F2E8E2D8D2C8C2B852EDC
:101F5E0008021FE2D201D204807AD2018076D20525
:101F6E00D2118070D205D20A806AAF28123C7D74DD
:101F7E002D2528F9E43461FA7B01C0031B8B3275E1
:101F8E003300753400E4F535D0031221D18F2E8E37
:101F9E002D8D2C8C2B852E0F803AAF28123C7D7404
:101FAE002D2528F9E43461FA7B01C0031B8B3275B1
:101FBE003300753400E4F535D0031221D18F2E8E07
:101FCE002D8D2C8C2B852E0D800AE4F52AF52905F6
:0A1FDE0028021DDF0527021DB622B0
:1032D0007BFF7A0E79F21218239069AEE0FEA3E02C
:1032E000FFC3E49FFFE49EFEAB07FA3395E0F9F8D5
:1032F0007F007E8C7D0A7C00121BB18F328E318D57
:10330000308C2F7BFF7A0F792E1218237BFF7A0FD8
:103310007986A210E433F52F1218237BFF7A0F79F8
:10332000BC850A2F1218237BFF7A0F79E8A209E4E3
:1033300033F52F1218237BFF7A107909A201E433A9
:10334000F52F1218237BFF7A107932A204E433F5AB
:103350002F1218237BFF7A107959A211E433F52F2D
:103360001218237BFF7A107984A20AE433F52F1216
:03337000182322FD
:102B55007E107FB2123639EF4E70037F01227E1050
:102B65007FB5123639EF4E602312391EA804A90528
:102B7500AA06AB077F007E8C7D0A7C00121BB11272
:102B85001C439069AEEEF0A3EFF0800A9069AE7435
:102B9500FFF0A374B8F07E107FBB123639EF4E609C
:102BA5000C123D45EF24D024FF92108002C2107E06
:102BB500107FC1123639EF4E600712391E8F0A8019
:102BC50003E4F50A7E107FC7123639EF4E600C120A
:102BD5003D45EF24D024FF92098002C2097E107F73
:102BE500CD123639EF4E600C123D45EF24D024FF4F
:102BF50092018002C2017E107FD3123639EF4E60FA
:102C05000C123D45EF24D024FF92048002C2047EBD
:102C1500107FD9123639EF4E600E123D45EF24D0A4
:102C250024FF920592118004C205C2117E107FE037
:102C3500123639EF4E600E123D45EF24D024FF9237
:0C2C450005920A8004C205C20A7F00222A
:10316C00C203C215C208C202C20FE4F5109066A1D8
:10317C00F0F50EF551C200D297D296750CFF906700
:10318C00ADF075080CC206C21490669F7409F0A3CA
:10319C00F0750F05C209C204C201C212C210D20CD2
:1031AC00E4F50AF509D2139069AE74FFF0A374B874
:1031BC00F0C20AC205C211E4F50D122B55EF6003E3
:1031CC00121D8EE49067A2F0C2ADF5C9D2CDD2CC5F
:1031DC00C2C9C2CAF5CDF5CC9069AEE0F5CBA3E07F
:1031EC00F5CA85CBCD85CACCE4F59830010C200905
:1031FC00095387BFD29FD29E8002D29E438740C282
:10320C009FC2ACC298C29975B81075B710D2CAD209
:04321C009CD2AC2272
:103D5F00E5136FFF90127A936512F513EF90117AB6
:043D6F0093F5122294
:013DEB0022B5
:1027F6008E288F29E4F52AF513F512AA06A9077B78
:10280600018B2E8A2F89309067A2E0121B63740118
:102816002530F530E4352FF52F30050F9067A3E00E
:10282600AB2EAA2FA930121B63800D9066A0E0ABD9
:102836002EAA2FA930121B63752E0185282F8529F4
:10284600300D0DE4FEEEC39D5018AB2E0530E5307D
:10285600AA2F7002052F14F9121B1DFF123D5F0EE1
:1028660080E3AB2E0530E530AA2F7002052F14F950
:10287600E513121B63AB2EAA2FA930E512121B63B8
:102886000D0D752C68752DAE752E0185282F8529A1
:1028960030852D82852C837402F0052DE52D70027E
:1028A600052C052AE4FEEEC39D504EAB2EAA2FA999
:1028B60030121B1DF52B6402600BE52B64036005CB
:1028C600E52BB40913852D82852C837409F0052D1B
:1028D600E52D7002052C052A852D82852C83E52B96
:1028E600F0052DE52D7002052C052A74012530F51D
:1028F60030E4352FF52F0E80AD852D82852C83741F
:1029060003F0052DE52D7002052C052A906693E04F
:10291600FCA3E0FDA3E0FEA3E0FFE4FAF9F8EF2450
:1029260001FFEA3EFEE93DFDE83CFC906693121C81
:102936006230240D7E107FE77C687DAEAB2A1229BB
:042946004AAF2A2248
:1030B000E4FF9066A0E0FE7D000FED2405F582E4BC
:1030C0003461F583EEF00F74052401F582E4346178
:1030D000F583E4F07C667D92FEED1DAA0470011C70
:1030E000F5828A83E0FBAA070F74052AF582E4348F
:1030F00061F583EBF00EBE04E07C667D96E4FEEDA8
:103100001DAA0470011CF5828A83E0FBAA070F74D4
:10311000052AF582E43461F583EBF00EBE04E07C11
:10312000667D9AE4FEED1DAA0470011CF5828A8377
:10313000E0FBAA070F74052AF582E43461F583EBFE
:10314000F00EBE04E07C667D9EE4FEED1DAA0470D8
:10315000011CF5828A83E0FBAA070F74052AF58219
:0C316000E43461F583EBF00EBE04E022C5
:083DDB00C2992099FDD2992242
:093DD200D2CAD29CD2ACC2082274
:103B9400AD077E677FA21227F69066A1EFF0D203ED
:103BA400E4F51030240D7E107FF67C687DAEE0FBDA
:103BB40012294AC296301003D20022E50A6003F5A6
:063BC4004E22123DDB223F
:103A2D008F2730030F30244E7E117F02E4FBFDFC07
:103A3D0012294A22906378E09066A0F0300C117E36
:103A4D00637F77E52724FCFD1227F69066A1EFF042
:103A5D00A21182055005750B05D214E4F510D203A1
:103A6D00C296301004D200800BE50A6004F54E803A
:073A7D0003123DDBC215221C
:10237500200603300B037F00222008030224FEC23F
:1023850008E4906475F09067ACE0FF547F24FCF599
:1023950027906476F090667AE0906477F0EF548049
:1023A500FF24AFF582E43467F583E0906478F07438
:1023B500AE2FF582E43467AD82FCE4F513F512FE29
:1023C5009067ACE0547FF9EEC39950140DEDAA0463
:1023D50070010C14F5828A83E0FF123D5F0E80E0E8
:1023E500E512451360443024197E117F109067ACC7
:1023F500E0548024AEF582E43467AD82FCAB011273
:10240500294A906697E0FCA3E0FDA3E0FEA3E0FF68
:10241500E4FAF9F8EF2401FFEA3EFEE93DFDE83C68
:10242500FC906697121C620224FE3005249067AC6E
:10243500E05480FF24AEF582E43467F583E09067CD
:10244500A2F074AF2FF582E43467F583E09067A3BB
:10245500F0E5277039C214F50B9067A3E0B4E01ED0
:102465007490F02005030224FED2062024030224E2
:10247500FE7E117F1FE4FBFDFC12294A807B302480
:10248500787E117F35E4FBFDFC12294A806B90674D
:10249500ACE0548024B0F582E43467F58363A2018F
:1024A50090647963A201AF271220C330241C7E11EA
:1024B5007F3E9067ACE0FB548024AEF582E4346740
:1024C500AD82FCEB547FFB12294A90668FE0FCA39A
:1024D500E0FDA3E0FEA3E0FFE4FAF9F8EF2401FF35
:1024E500EA3EFEE93DFDE83CFC90668F121C62A2C7
:1024F5000A82055002D206D216301605C2167F0191
:04250500227F00220F
:05001E00C2AEC2AC22DD
:103A8400300008209705C200123DDBE54EB4010664
:103A9400E4F54E123DDB302523C225E509600BD544
:103AA4000908630E80530E80C20230110FE50B60CB
:103AB4000BD50B08E4F510D203750B05A20A820698
:0F3AC400500C200309E4FF123B94C206D20B22E0
:0E3D9200301508201405C2157F01227F002283
:1039D4009080007480F090633663A201F583F582D1
:1039E40063A2017F081220C390633E63A20190800A
:1039F4008863A2017F0A1220C3908092E4F0A3742A
:103A040032F0A37401F0906348E0FF9080B1F0902D
:103A140080E1EFF09080957455F0A3F090800074ED
:093A240001F090800974F0F02219
:1037C700908009E04410F09080A0E0706C9080A198
:1037D7007482F09080A874FFF0A3F0A3F0A3F07FA9
:1037E700039080AEEFF07FCBA3EFF07F039080AC28
:1037F700EFF0A374CBF09080007402F09069B412DC
:103807001C6E000000009069B4E0908040F0906961
:10381700B5E0908041F09069B6E0908042F0906901
:10382700B7E0908043F0A3E4F0A3F0A3F0A3F090F7
:0A3837008018F0A3F0A3F0A3F02224
:1038BB00908009E04440F09080D17482F09063498D
:1038CB00E0FF9080DEF090634AE0FF9080DFF090A5
:1038DB0080027402F09069B8121C6E000000009018
:1038EB0069B8E0908058F09069B9E0908059F090F9
:1038FB0069BAE090805AF09069BBE090805BF0A3CE
:10390B00E4F0A3F0A3F0A3F0908030F0A3F0A3F0C9
:03391B00A3F022F4
:10384100908009E04420F09080B8E0706C9080B9DD
:103851007482F07F039080C6EFF07FCDA3EFF07FFD
:10386100039080C4EFF0A374CDF09080C074FFF09A
:10387100A3F0A3F0A3F09080017402F09069BC1250
:103881001C6E000000009069BCE090804CF09069D3
:10389100BDE090804DF09069BEE090804EF090695F
:1038A100BFE090804FF0A3E4F0A3F0A3F0A3F09069
:0A38B1008024F0A3F0A3F0A3F0229E
:103743008C278D28A907EAFDE975F018A424ACFF9E
:10375300E5F034808F82F583EDF0EBFDE975F01829
:10376300A4FFAEF024ACFBEE34808B82F583A3ED93
:10377300F08528828C83E0FDEF24A8FFEE3480FEE1
:103783008F82F583EDF08528828C83A3E08F828E70
:1037930083A3F0852882852783A3A3E0FDE975F041
:1037A30018A424A8FFE5F03480FE8F82F583A3A339
:1037B300EDF08528828C83A3A3A3E08F828E83A35D
:0437C300A3A3F022AA
:10352B008D2CAB07AA06908000E030E507906578FC
:10353B007401F0229069B4E0FCA3E0FDA3E0FEA3CC
:10354B00E0F5308E2F8D2E8C2DAE02AF038E838F38
:10355B008263A201E52F540744C0F5838530826353
:10356B00A201AF2C122135E4FCFDFEE530252CF534
:10357B0030EE352FF52FED352EF52EEC352DF52DB7
:10358B00908040E52DF0A3E52EF0A3E52FF0A3E509
:10359B0030F09080007420F0AF30AE2FAD2EAC2DFC
:0735AB009069B4121C6222BA
:1035B2008D27AB07AA06908002E030E50790657878
:1035C2007403F0229069B8E0FCA3E0FDA3E0FEA33F
:1035D200E0F52B8E2A8D298C28AE02AF038E838FC5
:1035E2008263A201E52A540744D0F583852B8263C6
:1035F200A201AF27122135E4FCFDFEE52B2527F5BC
:103602002BEE352AF52AED3529F529EC3528F52852
:10361200908058E528F0A3E529F0A3E52AF0A3E578
:103622002BF09080027420F0AF2BAE2AAD29AC288B
:073632009069B8121C62222E
:103220008F27908001E030E5099065787402F07F87
:1032300000229069BCE0FCA3E0FDA3E0FEA3E0F562
:103240002B8E2A8D298C2890667B63A201E52A5457
:103250000744C8F583852B8263A2017F0612214BA8
:10326000E52B2406F52BE4352AF52AE43529F52942
:10327000E43528F52890657963A201E52A540744CE
:10328000C8F583852B8263A201AF2712214BE4FC92
:10329000FDFEE52B2527F52BEE352AF52AED352900
:1032A000F529EC3528F52890804CE528F0A3E52990
:1032B000F0A3E52AF0A3E52BF09080017420F0AF95
:1032C0002BAE2AAD29AC289069BC121C62AF272214
:102A51009081E0E0F52705270527052705270527AC
:102A610005270527052705270527908010E0F52A6A
:102A7100A3E0F52BA3E0F52CA3E0F52D9081E1E097
:102A8100F5270527052705270527052705270527F5
:102A9100052705270527908014E0F52EA3E0F52FE3
:102AA100A3E0F530A3E0F531E530B52C08E531B50B
:102AB1002D037F0022E4F527E530540744E0F58338
:102AC10085318263A20190637563A2017F0812219F
:102AD1007B90637763A2019062AE63A2017F0612CD
:102AE10020C3906375E0F528A3E0F529E4F527906C
:102AF1006375E0702AA3E024F8F527E53054074414
:102B0100E0F58385318274082582F582E43583F509
:102B11008363A20190637563A201AF2712217BAE8B
:102B210028E4FCFDE5312529F531E5303EF530EDB0
:102B3100352FF52FEC352EF52E908014E52EF0A3D0
:102B4100E52FF0A3E530F0A3E531F090800074406B
:042B5100F0AF272298
:102509009081E6E0F52705270527052705270527F3
:1025190005270527052705270527908028E0F52A9F
:10252900A3E0F52BA3E0F52CA3E0F52D9081E7E0DE
:10253900F527052705270527052705270527052742
:1025490005270527052790802CE0F52EA3E0F52F18
:10255900A3E0F530A3E0F531E4F527E530B52C0A21
:10256900E531B52D05C21F022675E530540744F043
:10257900F58385318263A20190637563A2017F08A7
:1025890012217B906375E0F528A3E0F529E529453B
:102599002870099080027410F07F0022906682E012
:1025A900FFF46030906377E06F600302263C906629
:1025B90083E0FF906378E06F7079906684E0FF9024
:1025C9006379E06F706D906685E0FF90637AE06FE4
:1025D9006031805F906377E0906682F0906378E085
:1025E900906683F0906379E0906684F090637AE076
:1025F900906685F090637BE0FFA3E0906349CFF09C
:10260900A3EFF0906375E0702AA3E024F8F527E5BD
:1026190030540744F0F58385318274082582F582A8
:10262900E43583F58363A20190637563A201AF2743
:1026390012217BAE28E4FCFDE5312529F531E53091
:102649003EF530ED352FF52FEC352EF52EAF2DAEAD
:102659002CAD2BAC2AAB31AA30A92FA82ED3121C32
:102669005140099080027410F07F002290802CE57F
:102679002EF0A3E52FF0A3E530F0A3E531F090802B
:07268900027440F0AF2722AC
:102690009081E3E0F527052705270527052705276E
:1026A0000527052705270527052790801CE0F52A23
:1026B000A3E0F52BA3E0F52CA3E0F52D9081E4E059
:1026C000F5270527052705270527052705270527BA
:1026D000052705270527908020E0F52EA3E0F52F9C
:1026E000A3E0F530A3E0F531E4F527E530B52C0A99
:1026F000E531B52D05C2200227DBE530540744E85B
:10270000F58385318263A20190600463A2017F0E8C
:10271000122191906004E0F528A3E0F52990600C67
:10272000E0FFF4604590667BE0FEEF6E706EA3E024
:10273000FF90600DE06F706490667DE0FF90600E2A
:10274000E06F705890667EE0FF90600FE06F704C15
:1027500090667FE0FF906010E06F7040906680E0D0
:10276000FF906011E06F60048032D2D9906004E085
:10277000702AA3E024F2F527E530540744E8F583F6
:10278000853182740E2582F582E43583F58363A258
:102790000190600463A201AF27122191AE28E4FCEE
:1027A000FDE5312529F531E5303EF530ED352FF5E4
:1027B0002FEC352EF52EAF2DAE2CAD2BAC2AAB3138
:1027C000AA30A92FA82ED3121C515006E52945285E
:1027D00070099080017410F07F0022908020E52E17
:1027E000F0A3E52FF0A3E530F0A3E531F0908001F0
:0627F0007440F0AF272247
:102D42008E2C8F2D908000E030E50790657874011D
:102D5200F0229069B4E0FCA3E0FDA3E0FEA3E0F55D
:102D6200338E328D318C30E533FFE5325407FEE489
:102D72002FF52FEE34C0F52E852F82F5837423F0C4
:102D8200052FE52F7002052E532EC7F582852E835F
:102D9200740AF0052FE52F7002052E532EC790639B
:102DA2003E63A201852E83852F8263A2017F0612D4
:102DB20021357406252FF52FE4352EF52E852C832B
:102DC200852D8263A201852E83852F8263A2011243
:102DD2002119E4FCFDFE9069B4E0F8A3E0F9A3E058
:102DE200FAA3E02FFFEE3AFEED39FDEC38FCEF24BA
:102DF20008FFE43EFEE43DFDE43CFC9069B4121C95
:102E0200629069B4E0908040F09069B5E0908041B2
:102E1200F09069B6E0908042F09069B7E09080430C
:082E2200F09080007420F02202
:10294A008E318F328C338D348B35908000E030E5B8
:10295A00079065787401F0229069B4E0FCA3E0FD69
:10296A00A3E0FEA3E0F53B8E3A8D398C38E53BFFB8
:10297A00E53A5407FEE42FF537EE34C0F5368537CD
:10298A0082F5837423F00537E5377002053653362E
:10299A00C7F582853683740AF00537E53770020574
:1029AA00365336C790633E63A201853683853782E4
:1029BA0063A2017F0612213574062537F537E435FF
:1029CA0036F53685318385328263A2018536838561
:1029DA00378263A2011221198F3CEF2537F537E4BC
:1029EA003536F536E535601785338385348263A23B
:1029FA000185368385378263A201AF35122135E519
:102A0A003C24082535F535FFE4FCFDFEE53B2FF5B2
:102A1A003BEE353AF53AED3539F539EC3538F538D6
:102A2A00908040E538F0A3E539F0A3E53AF0A3E554
:102A3A003BF09080007420F0AF3BAE3AAD39AC3831
:072A4A009069B4121C622226
:102F0B008E458F468D47908000E030E507906578C1
:102F1B007401F0229069B4E0FCA3E0FDA3E0FEA3F2
:102F2B00E0F54D8E4C8D4B8C4AE54DFFE54C54072F
:102F3B00FEE42FF549EE34C0F548854982F58374DC
:102F4B0023F00549E549700205485348C7F58285CA
:102F5B004883EBF00549E549700205485348C79093
:102F6B00633E63A20185488385498263A2017F0684
:102F7B0012213574062549F549E43548F548854550
:102F8B008385468263A20185488385498263A201BA
:102F9B00AF4712213574082547F547FFE4FCFDFECA
:102FAB00E54D2FF54DEE354CF54CED354BF54BEC2A
:102FBB00354AF54A908040E54AF0A3E54BF0A3E58E
:102FCB004CF0A3E54DF09080007420F0AF4DAE4C6B
:0B2FDB00AD4BAC4A9069B4121C62229E
:1036BE008F40908000E030E5079065787401F0222D
:1036CE009069B4E0FCA3E0FDA3E0FEA3E0F5448E18
:1036DE00438D428C41E544FFE5435407FEE42FFF42
:1036EE00EE34C09062B463A201F5838F8263A201AF
:1036FE00AF40122135E4FCFDFEE5442540F544EED5
:10370E003543F543ED3542F542EC3541F5419080B8
:10371E0040E541F0A3E542F0A3E543F0A3E544F014
:10372E009080007420F0AF44AE43AD42AC4190693E
:05373E00B4121C622220
:102E2A008E278F28AB05908000E030E50790657803
:102E3A007401F0229069B4E0FCA3E0FDA3E0FEA3D4
:102E4A00E0F52E8E2D8D2C8C2BE52EFFE52D5407CB
:102E5A00FEE42FF52AEE34C0F529852A82F583741B
:102E6A0023F0052AE52A700205295329C7F5828528
:102E7A002983EBF0052AE52A7002052990633E634F
:102E8A00A201852983852A8263A2017F0612213540
:102E9A007406252AF52AE43529F5295329C7E52791
:102EAA00852A82852983F0052AE52A700205295395
:102EBA0029C7F582852983E528F0052AE52A7002C3
:102ECA0005295329C7E52E240AF52EE4352DF52DBB
:102EDA00E4352CF52CE4352BF52B908040E52BF0CE
:102EEA00A3E52CF0A3E52DF0A3E52EF09080007465
:102EFA0020F0AF2EAE2DAD2CAC2B9069B4121C6213
:012F0A0022A4
:0B3DC700E4FEEEC39F50030E80F822C4
:10337300E4F527E5272401FFE433FE123B1A7436F4
:103383002527F582E43463F583EFF00527E527C3AA
:10339300943F40DFE4F527E527247FFFE433FE1263
:1033A3003B1A742D2527F582E43461F583EFF0741D
:1033B3002D2527F582E43461F583E0FF6003B4FF34
:1033C3001D742D2527F582E43461F5837420F07490
:1033D3002E2527F582E43461F583E4F0800905277F
:1033E300E527C3948040B0E49061ACF0F527AF27A4
:1033F3007E00123B1A74AD2527F582E43461F58310
:0C340300EFF00527E527C394FE40E3220C
:103CEC00E4FDFCC3ED9FEC9E5015E4FBFA0BBB000E
:103CFC00010ABA01F8BB90F50DBD00010C80E4225D
:0D3DA0004390014390025390FE5390FD228A
:0D3DAD005390FD5390FE439002439001227D
:0F3D83005390FD439002E5905408FF5390FD22AA
:0D3DBA005390FD4390014390025390FD2271
:073DE300AE071FEE70FA228B
:103BFE00AD07E4FC5390FDEDA804088002C333D852
:103C0E00FC30E70543900180035390FE7F05123D83
:0C3C1E00E34390020CBC08DC5390FD2234
:103C5400E4FF5390FD7E07439002E59030E00D743D
:103C640001A806088002C333D8FC42075390FD1E06
:093C7400C3EE6480948050DF224D
:103C2A00AB05AA07123DA07FA0123BFE123D83AF4F
:103C3A0002123BFE123D83AF03123BFE123D83127A
:0A3C4A003DAD7F0A7E00123CEC2223
:103B1A00AB07AA06C3EB94FFEA9400400DE42BF529
:103B2A008274773AF583E493FF22123DA07FA012B4
:103B3A003BFE123D83AF03123BFE123D83123DA0B2
:103B4A007FA1123BFE123D83123C54123DBA123D34
:023B5A00AD229A
:103BCA008B2CA2AF9227C2AF85A22D53A2FE8E8361
:103BDA008F8205A28C838D8274091221BFE52C5332
:103BEA00A2FE43A2201221C153A2DF852DA2A22741
:043BFA0092AFFF2265
:103D0C00A2AF9227C2AF8C838D82EF1221BF43A248
:0D3D1C00201221C153A2DFA22792AFFF2287
:103CA4008F27A2AF9227C2AFE4F5838D82740612E8
:103CB40021BFE52743A2201221C153A2DFA22792EC
:043CC400AF7F0122AB
:103CC8008F27A2AF9227C2AFE4F5838D82740A12C0
:103CD80021BFE52743A2201221C153A2DFA22792C8
:043CE800AF7F012287
:101FE800A907E7FFA805EF93C3966008403B74FC78
:101FF8002FFF80F00F08EF93C3966008402B74FB07
:102008002FFF80E00F08EF93C3966008401B74FA17
:102018002FFF80D00F08EF93D3966008400B74F918
:102028002FFF80C01F1F1F1F1FEF54FEF80303F769
:10203800E893FC08E893FD08E893FE08E893FF227C
:1020480009E993C39D6008402974FB29F980F109C7
:10205800E993C39E6008401A74FA29F980E209E9F5
:1020680093D39F6008400B74F929F980D319191983
:102078001919E9C313C313FF22740093F8ECC3982A
:102088004024701F740193F8EDC3984019701474BC
:102098000293F8EEC398400E7009740393F8EFC3E7
:1020A8009840037F00227F0122EDF8E6F008A3DFC5
:1020B800FA22EDF8E0F608A3DFFA22E0A363A20112
:1020C800F0A363A201DFF475A2002263A201F0A3CA
:1020D80063A20122E0A363A201F0A363A201E0A32B
:1020E80063A201F0A363A201E463A201F0A363A2C7
:1020F80001DFE175A20022E0A363A2016DFE936CEB
:10210800FDEE058393FC158363A201DFEA75A20047
:10211800227F00E493A363A201F00F600CA3E58380
:10212800C2E3F58363A20180EA75A20022E0A363FB
:10213800A201F0A3E583C2E3F58363A201DFEE7594
:10214800A20022E0A363A201F0A3E583C2E4D2E3E4
:10215800F58363A201DFEC75A20022E0A363A2016C
:10216800F0A3E58344F8C2E5F58363A201DFEC75CB
:10217800A20022E583C2E3F583E0A363A201F0A3F2
:1021880063A201DFEE75A20022E583C2E4D2E3F583
:1021980083E0A363A201F0A363A201DFEC75A200B0
:1021A80022E58344F8F583E0A363A201F0A363A2C8
:1021B80001DFEE75A20022F922C002C004C0061297
:0921C800FFF0D006D004D0022281
:1034AB000208CCE493A3F8E493A34003F68001F263
:1034BB0008DFF48029E493A3F85407240CC8C33322
:1034CB00C4540F4420C8834004F456800146F6DFF1
:1034DB00E4800B0102040810204080903D29E47E1B
:1034EB00019360BCA3FF543F30E509541FFEE493E6
:1034FB00A360010ECF54C025E060A840B8E493A3AD
:10350B00FAE493A3F8E493A3C8C582C8CAC583CAD7
:10351B00F0A3C8C582C8CAC583CADFE9DEE780BE8F
:013D4400007E
:101B1D00BB010689828A83E0225002E722BBFE02C6
:091B2D00E32289828A83E49322F9
:101B3600BB010CE58229F582E5833AF583E0225064
:101B460006E92582F8E622BBFE06E92582F8E222AE
:0D1B5600E58229F582E5833AF583E49322C8
:101B6300BB010689828A83F0225002F722BBFE0161
:021B7300F3225B
:101B750075F008758200EF2FFFEE33FECD33CDCC27
:101B850033CCC58233C5829BED9AEC99E5829840AA
:101B95000CF582EE9BFEED9AFDEC99FC0FD5F0D687
:101BA500E4CEFBE4CDFAE4CCF9A88222B800C1B9B1
:101BB5000059BA002DEC8BF084CFCECDFCE5F0CBEF
:101BC500F97818EF2FFFEE33FEED33FDEC33FCEB28
:101BD50033FB10D703994004EB99FB0FD8E5E4F9E3
:101BE500FA227818EF2FFFEE33FEED33FDEC33FCD0
:101BF500C933C910D7059BE99A4007EC9BFCE99AC4
:101C0500F90FD8E0E4C9FAE4CCFB2275F010EF2F08
:101C1500FFEE33FEED33FDCC33CCC833C810D70708
:101C25009BEC9AE899400AED9BFDEC9AFCE899F843
:0E1C35000FD5F0DAE4CDFBE4CCFAE4C8F922D6
:0E1C4300C3E49FFFE49EFEE49DFDE49CFC22B2
:101C5100EB9FF5F0EA9E42F0E99D42F0E89C45F0E9
:011C61002260
:0C1C6200ECF0A3EDF0A3EEF0A3EFF022F5
:101C6E00A8828583F0D083D082121C85121C851227
:101C7E001C85121C85E473E493A3C583C5F0C5834C
:101C8E00C8C582C8F0A3C583C5F0C583C8C582C8C0
:011C9E002223
:1017C100E53B242FF8E6053B22782C302E02782FBA
:1017D100E475F001121CEE021B1D2027EB7F2ED2B7
:1017E100278018EF540F2490D43440D4FF302B0BB2
:1017F100EF24BFB41A0050032461FFE53C600215D9
:101801003C053FE53F7002053E302E0D782CE47516
:10181100F001121CEEEF021B63023AD37403D22EC5
:101821008003E4C22EF53B8B2C8A2D892EE4F53CF6
:10183100F53EF53FE53C60077F201217FC80F5750A
:101841003DFFC228C227C229C22AC22CC22DC22FE3
:101851001217CAFF700D302E057F0012180DAF3F11
:10186100AE3E22B4255FC2D5C22B1217CAFF24D0C7
:10187100B40A00501A75F00A783C30D50508B6FF55
:101881000106C6A426F620D5047002D22A80D924E6
:10189100CFB41A00EF5004C2E5D22B021A0DD228A0
:1018A10080C6D22780C0D22980BCD2D580BAD22CA2
:1018B10080B47F201217FC2029077401B53C004039
:1018C100F11217C1FF1217FC021835D22FD22D8049
:1018D100951217C1FB1217C1FA1217C1F94A4B70C1
:1018E1000679DE7A1A7BFF20292EE53C602A7E00EC
:1018F1008E82758300121B3660060EEE653D70F018
:10190100C2D5EBC0E0EAC0E0E9C0E0EE121A54D063
:10191100E0F9D0E0FAD0E0FB121B1DFF60AAEBC09A
:10192100E0EAC0E0E9C0E01217FCD0E02401F9D000
:10193100E03400FAD0E0FBE53D0460DCD53DD98020
:10194100877BFF7A1A7950D229809C79108002799D
:1019510008C22DC22F8008D2D5790A8004790AC223
:10196100D5E53D047002F53DE4FAFDFEFF1217C115
:10197100FC7B082028131217C1FD7B1030270A12A7
:1019810017C1FE1217C1FF7B20EC3382D592D550CF
:1019910013C3E43027069FFFE49EFEE42028039D45
:1019A100FDE49CFCE4CBF8C228EC700CCFCECDCC8E
:1019B100E824F8F870F38017C3EF33FFEE33FEED40
:1019C10033FDEC33FCEB33FB994002FB0FD8E9EB21
:1019D100302805F8D0E0C448B228C0E00AEC4D4EEA
:1019E1004F78207B0070C2EAB53D0040BCC0E012D8
:1019F1001A56D0F0D0E0202804C4C0E0C4B228C0F8
:101A0100F01217E5D0F0D5F0EB021835121D4D1884
:101A1100D253194C5818A34C189F4219504F1958BA
:0F1A21004419584918B843195E551942461942DD
:101A3000451942471AFE5018A72D18AB2E18CE2B69
:101A400018AF2318CC201AE72A186748000018C6D8
:101A50003F3F3F00790AA2D5202A14302C09B91043
:101A6000020404B9080104A2D5202D02500104206B
:101A700029689229B53C005034C0E07F20302A19F3
:101A80007F30A229722D722C500F121AADC229C2BA
:101A90002DC22CC22F7F30800F302C03E9C0E01202
:101AA00017FC302C03D0E0F9D0E0B53CCC302C173B
:101AB0007F30B9100C1217FC7F58302B077F7880CD
:101AC00003B908031217FC3029057F2D0217FC7F8C
:101AD00020202FF87F2B202DF322922980CF286EF3
:101AE000756C6C2900D2281217C13028F8C22878EA
:101AF0003C30D50108F60218672D5043495812179B
:101B0000C12403B405004001E4901AF9931217EDC3
:0D1B1000743A1217EDD22A753C0402194CEC
:1021D1008B2F8A308931E4F53BF53AF539F538F53D
:1021E10036F537E533453445326012EBC0E0EAC0DD
:1021F100E0E9C0E0AB32AA33A934121CFEAB2F05D3
:1022010031E531AA307002053014F9121B1DF53C7D
:10221100C394094007E53CD3940D40E1E53C6420BB
:1022210060DBE53CB42D054337038016E53CB42B58
:1022310005433701800C74FF2531F53174FF3530CA
:10224100F530E53560046410703FAB2FAA30A93139
:10225100121B1D64306009E535702E75350A802921
:10226100900001121B36FF64786004EFB4581343E9
:10227100370175351074022531F531E43530F5300B
:102281008007E5357003753508AB2F0531E531AAB7
:10229100307002053014F9121B1DF53CC3946140E6
:1022A1000AE53CD3947A5003533CDF74D0253CF5C6
:1022B1003CC3940A400CE53C9411406D74F9253CF3
:1022C100F53CE53CD395355060433701853B40856E
:1022D1003A3F85393E85383DAF357E00E4FCFDABA4
:1022E1003BAA3AA939A838121C9FC8ECC8C9EDC944
:1022F100CAEECACBEFCBE4FCFDFEEB253CF53BEE91
:102301003AF53AED39F539EC38F538AF3BAE3AAD3F
:1023110039FCAB40AA3FA93EA83DD3121C51500342
:1023210002228A43370402228AE53720E003E4804F
:102331002DE53345344532601EAB2FE53124FFF9DD
:10234100E53034FFFAEBC0E0EAC0E0E9C0E0AB32CF
:10235100AA33A934121CFEE53730E20774FFFFFEF1
:10236100FDFC22E537AF3BAE3AAD39AC3830E10385
:04237100021C4322E5
:101C9F00E88FF0A4CC8BF0A42CFCE98EF0A42CFCE4
:101CAF008AF0EDA42CFCEA8EF0A4CDA8F08BF0A462
:101CBF002DCC3825F0FDE98FF0A42CCD35F0FCEBC1
:101CCF008EF0A4FEA9F0EB8FF0A4CFC5F02ECD3986
:0F1CDF00FEE43CFCEAA42DCE35F0FDE43CFC22F3
:101CEE00FAE6FB0808E6F925F0F618E6CA3AF622F7
:101CFE00BB011A89828A83D0F0D0E0F8D0E0F9D007
:101D0E00E0FAD0E0FBE8C0E0C0F0021D7C5016E91E
:101D1E00F8D083D082D0E0F9D0E0FAD0E0FBC082D8
:101D2E00C083021D73BBFE16E9F8D083D082D0E0CB
:0F1D3E00F9D0E0FAD0E0FBC082C083021D8522FD
:101D4D00D083D082F8E4937012740193700DA3A325
:101D5D0093F8740193F5828883E473740293686039
:061D6D00EFA3A3A380DF39
:091D7300EBF608EAF608E9F62295
:091D7C00EBF0A3EAF0A3E9F02268
:091D8500EBF208EAF208E9F2228F
:00000001FF
